:10000000CAC20000E5C200000C946430E1C20000E6
:10001000DFC20000DDC20000DBC20000D9C2000068
:10002000D7C20000D5C200000C94992E0C94812FE9
:100030000C944E2ECDC20000CBC20000C9C20000FD
:10004000C7C20000C5C20000C3C20000C1C2000098
:10005000BFC200000C94752EBBC20000B9C20000E4
:10006000B7C20000B5C20000B3C20000B1C20000B8
:10007000AFC20000ADC20000ABC20000A9C20000C8
:10008000A7C20000A5C20000A3C20000A1C20000D8
:100090009FC200009DC200009BC2000099C20000E8
:1000A00097C2000095C2000093C20000050109023A
:1000B000A10185020901A1000509190129081500FE
:1000C0002501950875018102050109300931158165
:1000D000257F95027508810609381581257F9501D0
:1000E00075088106050C0A38021581257F95017572
:1000F000088106C0C005010980A101850319012AF4
:10010000B700150126B700950175108100C0050CD8
:100110000901A101850419012AA002150126A002E6
:10012000950175108100C00660FF0961A101096297
:10013000150026FF00952075088102096315002629
:10014000FF00952075089102C005010906A101056F
:100150000719E029E7150025019508750181029529
:1001600001750881010507190029FF150026FF0008
:100170009506750881000508190129051500250156
:10018000950575019102950175039101C00000006C
:10019000000000000000000000000000000000005F
:1001A000000000000000000000000000000000004F
:1001B000007E0F00D4FFFFFFC700000078000000A2
:1001C00000000000002A2B280000000000000000B2
:1001D000000000000000000029000000002C1E3478
:1001E00020212224342627252E362D3738271E1F7E
:1001F000202122232425263333362E37381F0405A9
:10020000060708090A0B0C0D0E0F10111213141516
:10021000161718191A1B1C1D2F3130232D350405F4
:10022000060708090A0B0C0D0E0F101112131415F6
:10023000161718191A1B1C1D2F3130354C09025B7B
:1002400000030100A0FA09040000010301010009F4
:100250002111010001224400070581030800010962
:100260000401000203000000092111010001222203
:100270000007058203200001070503032000010990
:100280000402000103000000092111010001227B8A
:10029000000705840320000112010002000000088D
:1002A000ABC239390100010203011C037600690069
:1002B00061006C003A0066003600340063003200D2
:1002C00062003300630000002203410072006300FB
:1002D00068006900740065007500740068006900BA
:1002E00073002000640075007800000010037400A3
:1002F0006100700069006F006B006900000004037A
:10030000090414001A000800150017000400160064
:10031000070009000A001D001B0006001900050067
:100320002B43E1000000000000001C0018000C003E
:10033000120013000B000D000E000F00340011001E
:1003400010003600370038002C0028410000000063
:1003500000001E021F02330033022D023100310261
:100360002F0226022F00000000003002270230007A
:10037000010022520000000000002E002400250091
:1003800026002E0225022100220023002D00270036
:100390001E001F00200038000100010000000000C6
:1003A00000001E141F1420142114BD00A800AA0070
:1003B000AE00A900BE00B000AC00AD00AB00000074
:1003C00001000100000000000000000024023500D0
:1003D0003502000000002102220223022D0200004B
:1003E0001E021F02200200000100010000000000A8
:1003F00000002900500409014F044900A452A852EA
:10040000A252A152B4521D011B0106012B00190179
:10041000010001000000000000004B004A005200F3
:100420004D0039004E00500051004F004C00280094
:100430002A00E400E20065000100245200000000F0
:10044000000000000000091346000000A452A8525A
:10045000A252A152B4521D131B1306132B021913DF
:1004600001000100000000000000450040004100C4
:100470004200000044003D003E003F0000004300F9
:100480003A003B003C0000000100010000000000B9
:100490000000FD377A585A000004E6D6B446020040
:1004A000210116000000742FE5A3E0013F00915DDB
:1004B000003D8889A654750A36E182AEFA7A1AA6FA
:1004C000FCA2ED495F2BD164DB9630A72B46AB9E97
:1004D000F559ECD5D368B65BFED1E16EC41BB98487
:1004E0001554A417CD6C9049895455A588012E5BED
:1004F0005BAF1340B078303009DFC39078351FDE32
:100500001802F7E77D47122C69FEF6D74D8F74F578
:1005100064447E0302197D127F6E9E47BFE050A2A5
:10052000E8A21FF25C57B453C529502385E6A861A1
:10053000490C8806A3E4C919DBD6071EE5672AAB78
:10054000C45600000000B890350CE8302CD90001EA
:10055000AD01C002000035C57E2EB1C467FB0200AC
:1005600000000004595A504F52514A4D4B4E2A4CEC
:100570002F30B6B7ABACBBBCA9AABDBECFD0CDCED9
:10058000DBDCD9DA0D0E0B0F1A0508050905071873
:1005900011130408120C11241FBECFEFDAE0DEBFE6
:1005A000CDBF11E0A0E0B1E0E6EEF5E602C00590B7
:1005B0000D92A83DB107D9F724E0A8EDB1E001C044
:1005C0001D92A63DB207E1F70E944C270C947532AC
:1005D00017CD9C01FB019A9581159F4120F5832F32
:1005E0008170B32FB270AA27732F74706627532FB0
:1005F0005870442734FF0DC08295807FAB2B09F0E3
:100600008062672B09F08064452B09F080680995AA
:100610000895AB2B09F08260672B09F08460452BAD
:10062000B1F38860F4CF80E0F2CF0C94C331089529
:10063000982F92959F7024E0911102C020E0982F8E
:10064000892F86958695811511F02E5F982F892F19
:100650008695820F08958093D20408958093D304E1
:10066000089521E030E001C0220F8A95EAF78091D9
:10067000D304822BF3CF21E030E0A90102C0440F64
:10068000551F8A95E2F7CA0180959091D30489237A
:10069000E5CF292F983090F5853080F590E035E052
:1006A000239F800D911D1124282F277041E001C048
:1006B000440F2A95EAF723E0969587952A95E1F766
:1006C000FC01EE0FFF1FE80FF91FE65FFC4F20E073
:1006D00030E070E05191DF01CB01022E02C096950F
:1006E00087950A94E2F78170819585278423852771
:1006F0008E932F5F3F4F2330310561F70895292FE7
:10070000983078F5853068F590E035E0239F800DCE
:10071000911D1124682F677023E0969587952A957F
:10072000E1F7FC01EE0FFF1FE80FF91FE65FFC4F3A
:1007300040E050E080E0219130E0062E02C0369586
:1007400027950A94E2F721703327042E01C0220F67
:100750000A94EAF7822B4F5F5F4F4330510559F7F8
:10076000089580E008959091D30421E030E0F901EC
:1007700001C0EE0F8A95EAF7D90102C0AA0FBB1F8C
:100780006A95E2F7EA2B01C0220F4A95EAF7892F12
:100790008E23E81303C0892F822B60CF2095822FF0
:1007A0008923FBCF8091B8029091B702981301C0C2
:1007B00008958F5F8770FACF90911E0480958923EA
:1007C00080931E04282F2770211110C0891771F003
:1007D0009091D50492FF0AC08695869586954BDF49
:1007E00010921E041092200410921F0408959091FC
:1007F0001B04982B90931B040895982F909580913B
:100800001B04892380931B04089580911A04811589
:1008100031F010921A0410922204109221040895CB
:10082000803E9105D9F1C8F48133910509F482C065
:1008300048F48932910509F472C08A32910509F4AD
:1008400080C0089589339105E9F082389105D1F08F
:100850008533910509F45EC00895843E9105D9F170
:1008600048F4823E910539F1833E910549F181EECC
:1008700090E00895863E9105C9F1873E910509F4FF
:100880003EC008952091D4042370211164C02091AA
:10089000D50423FF14C089E290E008952091D40488
:1008A00020FD45C03091D50430FF09C024FD24C08F
:1008B00083EE90E008952091D40422FDF7CF0895AF
:1008C0002091D40422FD44C03091D50430FD43C0B2
:1008D00024FFF5CF11C02091D50421FFF0CF8091E6
:1008E000D40484FD09C087EE90E008952091D404DB
:1008F00023FFE5CF24FFF7CF80E090E0089520911B
:10090000D40423FD2BC03091D50431FFE1CF84EE18
:1009100090E008952091D40425FFD1CFBCCF209141
:10092000D40425FD1EC02091D50423FFC8CF89E340
:1009300090E008952091D40426FFC1CF8AE290E090
:1009400008952091D40426FFBACF81E390E0089562
:1009500082EE90E0089580EE90E0089586EE90E0BB
:10096000089585E390E008959091D40492FF10C01B
:1009700041E0282F2471243009F040E031E0282F95
:100980002871283009F030E0431711F02CE082275D
:1009900093FF10C041E0282F2471243109F040E07A
:1009A00031E0282F2871283109F030E0431711F089
:1009B0002CE082273091D50430FF10C051E0282F61
:1009C0002171213009F050E041E0282F28712830B2
:1009D00009F040E0541711F029E0822731FF10C0E0
:1009E00041E0282F2171213109F040E031E0282F2A
:1009F0002871283109F030E0431711F029E08227EF
:100A000094FD877E08951F93CF93DF9309DFEC0158
:100A1000811522E5920708F052C0811540E5940740
:100A200008F0CDC0803E910520F58D3C910508F081
:100A3000A1C0883A910570F4853A910508F097C0F5
:100A400081309105B9F10497813A910598F1C0E0A0
:100A5000D0E030C0885A91094B97C8F7C85AD0E007
:100A6000CC0FDD1FC459DE4F0990D881C02DD4644E
:100A700021C0811550E49507B0F4C11580E2D80774
:100A800008F0B3C0C83ED105A8F0CE019A958115F3
:100A90009F41E8F68D2F68DF182FCE019927C0DE21
:100AA000EC01D12B07C09927BBDECC27DF70C82B08
:100AB000D92BD06ACE01DF91CF911F910895803854
:100AC00042E59407C8F5803652E5950708F05BC00B
:100AD000C03482E5D807D0F4C03292E5D90708F0D7
:100AE0004BC08C2F8695869520E2829FC0011124F1
:100AF000C37021E030E0A90102C0440F551FCA9520
:100B0000E2F7EA01C82BD92BDD68D4CF8C2F86956C
:100B10008695877050E2859FC0011124C37021E043
:100B200030E0A90102C0440F551FCA95E2F7EA015F
:100B3000C82BD92BDC68BECF803C52E5950758F412
:100B40008F71C03AD245A0F590E0982F8827EC012C
:100B5000C46FD06AAFCF805C9245809708F077CFA2
:100B6000DC2FCC27CC27DF71C06FD06AA3CFA4972E
:100B7000D064A0CFD0659ECFCF71D0E0DC2FCC2742
:100B8000C16FD06A97CF86958695877020E2829F45
:100B9000C0011124C37021E030E0A90102C0440F5C
:100BA000551FCA95E2F7EA01C82BD92BDA6882CF24
:100BB000DBDEC82FD0E0DC2FCC27D0627BCF8F715B
:100BC000D3DE93E0CC0FDD1F9A95E1F7CC27DF70E1
:100BD000282F30E084FF05C050E1859F900111244B
:100BE0003327C22BD32BD06965CF8D2F8F71BCDEFD
:100BF000182FCE01992714DEEC01D12BDECF80E037
:100C0000089581152CE7920741F4209189023091D3
:100C10008A02232B11F480E090E00895E0E9F3E0EC
:100C200080E090E06DED75E240E056E222E736E2CA
:100C300077836683518740873387228797878687A4
:100C4000019670968830910599F70895FB018115FA
:100C500020E2920728F4811541E0940738F40895C2
:100C60009C0130522115304348F00895392F94FFEC
:100C700002C03295307F2081232B2083992708954D
:100C8000462B22FF0FC0982F92959F708F70892B53
:100C9000962F92959F706F70692B942F92959F70ED
:100CA0004F70492B982F9623961309C050E040951A
:100CB000509590E04823592381E0452B09F080E0CE
:100CC00008951092640410926304E3E2F4E08581D5
:100CD000811102C014821682379684E0EB35F80742
:100CE000B1F70895AC013091660460916504232F3B
:100CF000621301C00895822F90E0FC01EE0FFF1FE8
:100D0000E55AFB4F0190F081E02DE417F50791F4CF
:100D100067E0649FF001659FF00D1124ED5DFB4FCE
:100D200041E044832313E6CF019683709927809393
:100D3000660408950196282F2370DACF0F931F932E
:100D4000CF9301E010E0082E01C0000F0A94EAF7EB
:100D5000C09119049C2F9023911115C090911E04ED
:100D6000969596959695891306C010921E0410923A
:100D7000200410921F0475DCC027C0931904CF9182
:100D80001F910F91089577DCF7CF282F35EB2303C0
:100D9000C001112497FF04C080589109892F08953C
:100DA00080589F4FFBCF80911B0380FD14C081FDB5
:100DB00014C082FD16C080911A03811581F08E3116
:100DC00080F420E5829FC00111246EE170E00E9452
:100DD000AA31862F089584E1089588E2089588E075
:100DE000089580E5089580911B0380FD17C081FD63
:100DF00017C082FD19C080911903811599F08832BE
:100E000098F428E0829FC001112468E270E00E94FB
:100E1000AA316115710551F0862F089562E0FCCF6B
:100E200064E0FACF61E0F8CF68E0F6CF81E00895A2
:100E30009091770389029001112437FF03C08093BA
:100E4000770308952F3731051CF4980F909377039B
:100E500008959C0180E090E0F901E80FF91FE4910A
:100E6000E41307C091E08927F901E80FF11D84918F
:100E700008950196861780F380E00895FA0130976F
:100E800009F0099508958091A102811569F0E0911A
:100E9000AD02F091AE02309739F00190F081E02D73
:100EA000309711F00995089580E00895A3E0B0E02F
:100EB000ECE5F7E00C9483319C018091080290915D
:100EC000090282179307B1F03093090220930802B8
:100ED000E091AD02F091AE02309761F00084F185AF
:100EE000E02D309739F083E089833B832A83CE015C
:100EF000019609952396E2E00C949F31A3E0B0E0BF
:100F0000E4E8F7E00C9483319C0180910602909113
:100F1000070282179307B1F030930702209306026D
:100F2000E091AD02F091AE02309761F00084F1855E
:100F3000E02D309739F084E089833B832A83CE010A
:100F4000019609952396E2E00C949F319C01FC01E7
:100F500032968FEF90E04191461751F08F3F19F490
:100F6000411101C0892F9F5F9630A9F78F3F09F487
:100F70000895280F311D87FD3A95F9016283089580
:100F80009C01FC013296285F3F4F8191861302C07D
:100F9000DF011E92E217F307C1F708958091010166
:100FA00008952FB7F8948091020290910302A091C6
:100FB0000402B09105022FBF0895962F2091D50409
:100FC00022FF0EC0682F660F660F660F692B6093B5
:100FD0001E0447DBE6DF9093200480931F040895EE
:100FE00040CB90911A04292F2823211559F0809580
:100FF000892380931A04811531F0D3DF8093210473
:1010000090932204089580E090E0F8CFCADF209109
:101010001E0330911F03232B211521F080937A02A8
:1010200090937B022091200330912103232B2115E3
:1010300021F08093780290937902E091AD02F091D3
:10104000AE02309759F00680F781E02D309731F0ED
:1010500082E080931C038CE193E00995089561156B
:1010600009F441C0E3E3E80FE33148F4F0E0E95864
:10107000FD4C0C94BD3197DE819580931F03C6CF44
:1010800092DEFBCF90DE819580931E03F8CF8BDE3E
:10109000FBCFA9DE80932003F2CFA5DE8195FACFA6
:1010A000A2DE819580932103EACF9DDEFBCF815D97
:1010B000990B21E030E001C0220F8A95EAF7809178
:1010C0001D03822B80931D03DACF80911B03816067
:1010D00080931B03D4CF80911B038260F9CF809152
:1010E0001B038460F5CF40911E038D3C59F4809121
:1010F0001F0387FF0DC010921F03411559F4109272
:101100001A0308C08E3C81F480911F0318169CF3CB
:10111000411581F08091200390912103892B811149
:10112000AECF10921903ABCF8F3C41F447FFF0CF05
:1011300010921E0380911F038115E0CF803D19F4AA
:101140001416B4F3E5CF90912003893D29F41916C4
:10115000FCF610922003DCCF8A3D19F497FFD8CF1C
:10116000F8CF909121038B3D29F497FFD1CF1092B6
:101170002103CECF8C3D19F41916CCF3C9CF9FE2D1
:10118000980F983090F4815D990B21E030E0B9011F
:1011900002C0660F771F8A95E2F7CB018095909188
:1011A0001D03892380931D03B3CF8D3D31F48091BE
:1011B0001B038E7F80931B03ABCF8E3D21F4809168
:1011C0001B038D7FF7CF8F3D09F0A2CF80911B03CA
:1011D0008B7FF0CF2FB7F8946091020270910302D9
:1011E00080910402909105022FBF08950F931F93E1
:1011F0008091A102811521F0EDDF1F910F910895DB
:10120000E9DF0091A3021091A4022091A502309180
:10121000A602600F711F821F931FEFCF87E797E72A
:10122000909301088093000888E19AE00FB6F89443
:10123000A895809360000FBE90936000FFCF089543
:10124000FC019B018091F8019091F90186179707A5
:1012500040F0672B29F48091E8008E778093E800B6
:10126000C90140E0009741F4411106C08091E800B7
:1012700082FF2FC080E0089520918B022115A9F1F3
:101280002530A9F12091E80023FD2DC02091E80030
:1012900022FDECCF2091E80020FFE4CF3091F30055
:1012A0002091F200009719F02830310558F041E004
:1012B0002830310509F040E02091E8002E77209396
:1012C000E800D0CF41914093F10001972F5F3F4F4D
:1012D000E9CF80918B02811541F0853041F08091FA
:1012E000E80083FFC3CF81E0089582E0089583E0A2
:1012F00008958091F20187FF13C08091E80082FF7A
:1013000006C08091E8008B778093E8000895809173
:101310008B028111F2CF089580918B028115D9F350
:101320008091E80080FFF8CF8091E8008E77ECCFC5
:101330002091E4003091E50095E6A9012091EC00B0
:10134000822F817020FF06C08091E80080FF06C0D8
:1013500080E008952091E80022FD1AC080918B0260
:10136000811589F0853089F08091EB0085FD0FC0F3
:101370002091E4003091E50042175307F9F29A9565
:10138000E1F684E0089582E0089583E0089581E025
:101390000895E8EDF0E080818E7F80831092E20076
:1013A0001092DA001092E100A0EEB0E08C91816022
:1013B0008C9380818F77808319BCA7EDB0E08C91EE
:1013C0008E7F8C9380818F7E80831092F1010895AF
:1013D000E091AD02F091AE02309739F00284F385CE
:1013E000E02D309711F060E209950895FC01AC0101
:1013F0004C5F5F4F8FEF61E39191892728E030E0E8
:10140000982F990F87FF09C0892F862721503040D8
:10141000B9F7E417F50781F70895892FF7CF982FCB
:101420009093E900891771F07091EC002091ED0024
:101430005091F00021FD09C09F5F973089F780939C
:10144000E9000895762F242F50E03091EB003E7F85
:101450003093EB003091ED003D7F3093ED00309103
:10146000EB0031603093EB007093EC002093ED00C3
:101470005093F0002091EE0027FDDECF0895A0E00C
:10148000B0E0E5E4FAE00C947D31C8EDD0E088816D
:101490008F7E8883E7EDF0E080818160808384E047
:1014A00082BF81E08093F10188818E7F888302EE84
:1014B00010E0F80110821092DA0081EEC82ED12CD3
:1014C000F601108288818F7788838881806888837D
:1014D00088818F7D888319BC10928B021092F00155
:1014E00010926E021092EF0190EEE92EF12CF701AE
:1014F00080818B7F808388818160888342E060E087
:1015000080E08DDFF60180818E7F8083F80180810D
:1015100081608083808188608083F70180818E7FF5
:101520008083888180618883CDB7DEB7E8E00C9442
:101530009931E091B8029091B70229E0E91302C015
:1015400080E00895AE2FB0E02E9FF0011124E75403
:10155000FD4F3181361306C03081381303C0358109
:10156000341304C0FD013196E770E8CF81E008959F
:101570000F931F93CF93DF938B01EA0190918B021E
:10158000943051F58093E9008FEF9091E80095FD3C
:1015900006C095ED9A95F1F700008A95B1F7809114
:1015A000E80085FF19C0C4DE811111C08091E800F8
:1015B00085FD06C08091E8008E778093E800F3CF28
:1015C000F80181918F018093F100219779F7809143
:1015D000E8008E778093E800DF91CF911F910F9103
:1015E0000895792F603229F440E250E0682F82E0BC
:1015F000BFCF0895CF93DF93D82FC92F48E050E095
:10160000682F792F81E0B4DF88E0ED2FFC2FAAEF5F
:10161000B1E001900D928A95E1F7DF91CF910895A5
:10162000BC0146E050E084E0A3CFBC0143E050E0C1
:1016300084E09ECFA0E0B0E0E0E2FBE00C947B31E0
:10164000F82EE92EB62EA72E8A018091EC019AE0A1
:10165000C92ED12C8A3018F0CC24C394D12CC1E0EF
:10166000D0E06B2D7A2D8F2D9E2DF80109958111DB
:1016700016C02196CC16DD0694F0CC9FC001CD9FFC
:10168000900D900D112420E030E045E34A95F1F7EC
:1016900000002F5F3F4F28173907B9F7E2CFCDB7CA
:1016A000DEB7EAE00C9497319091D50492FB2227A3
:1016B00020F9281771F080FB92F99093D50460917E
:1016C000D4047091D50484E090E00E945A3282E004
:1016D00073C80895609116048CE090E00C94403239
:1016E0001F93CF93DF93962F122F632F282F292B31
:1016F0002830C8F44530B8F4C42FD0E0CC0FDD1F3B
:101700002AE0929FC00DD11D112490E5899FC00D44
:10171000D11D1124CE0189960E944032612FCE0145
:101720008A960E944032DF91CF911F910895CF9306
:10173000DF93C0911B0480911D04C82B80911A0473
:101740008115E1F02EDC2091210430912204821BCE
:10175000930B8838934108F058D8D0911A0420E0B0
:101760008CED91E0FC013081019631112F5F31E069
:10177000823E9307B9F7211148D8CD2BC093DA01E7
:1017800048E050E06FEA72E08AED91E00E94F731A4
:10179000892BB9F088E0EAEDF1E0AFEAB2E0019020
:1017A0000D928A95E1F7E091AD02F091AE0230978B
:1017B00041F00280F381E02D309719F08AED91E03D
:1017C0000995DF91CF910895CF9310921B04C6E045
:1017D000ECEDF1E0DF018C2F1D928A95E9F780E0B6
:1017E00090E064DB80E090E089DB10921D049FDFD5
:1017F000ECE1F3E0DF011D92CA95E9F710921A03BC
:101800001092190310921B0301DCCF910895DCDFC5
:101810002FEF84E39CE0215080409040E1F700C02E
:10182000000088E19AE00FB6F894A89580936000D4
:101830000FBE90936000FFCFAAE2B0E0E2E2FCE0CE
:101840000C94823182EF91E0FC0101962091F1002D
:10185000208321E08A3F9207B9F78091F301893014
:1018600009F457C0C8F4823009F4B2C0833009F4D7
:1018700082C0813081F18091E80083FFE6C08091D1
:10188000F2019091F3019A3008F0DFC0E92FF0E007
:10189000E657FD4C0C94BD318A3009F489C08B3079
:1018A00051F78091F201813231F78091F6019091E8
:1018B000F701892B01F78091E800877F8093E8008A
:1018C00018DD81E09091F401911101C080E08093D6
:1018D00002017ADFD0CF8091F201813A61F68091E6
:1018E000E800877F8093E8008091F6019091F701EE
:1018F000892B59F060E080E090E070E0A1DC8091FD
:10190000E8008B778093E800B6CF68E08AEF91E03B
:10191000F4CF8091F201813209F0ADCF8091F601D0
:101920009091F7018D7F892B09F0A5CF8091E80078
:10193000877F8093E8008091E80082FF17C0909134
:10194000F3008091F200029731F48091F100813030
:1019500011F0863021F48091F10080930101809193
:10196000E8008B778093E800C4DC85CF80918B0200
:101970008111E1CF80CF8091F201813A09F07BCFD4
:101980008091F6019091F701892B09F074CF809135
:10199000E800877F8093E8008091E80080FFFCCF1B
:1019A000809102018093F1008091E8008E77DACF78
:1019B0008091F201813209F05ECF8091E800877F4B
:1019C0008093E80096DC8091F5018093000153CF6D
:1019D0008091F201813A09F04ECF8091E800877F33
:1019E0008093E8008091E80080FFFCCF80910001A7
:1019F000D9CF803889F0823841F58091F6018F7017
:101A0000873018F58093E9008091EB0085FB8827EB
:101A100080F91092E90006C080916E02880F9091C3
:101A2000EF01892B9091E800977F9093E8008093D5
:101A3000F1001092F1008091E8008E7723C08111AF
:101A400016C08091F401813009F18091E80083FF94
:101A50000AC08091E800877F8093E8008091EB00C6
:101A600080628093EB00AA96E3E00C949E31823072
:101A700061F78091F401811581F01092E900809165
:101A8000E800877F8093E80034DCDFCF81E093308B
:101A900009F080E080936E02F0CF8091F6018F70A4
:101AA0002FEF280F263088F68093E9002091EB0075
:101AB00020FFE3CF933031F48091EB00806280937C
:101AC000EB00DBCF9091EB0090619093EB0021E075
:101AD00030E0A90102C0440F551F8A95E2F74093F8
:101AE000EA001092EA008091EB008860E8CF811153
:101AF000ACCF1091F4011F778091E3008078812BA7
:101B00008093E3008091E800877F8093E800F1DB19
:101B10008091E80080FFFCCF8091E3008068809393
:101B2000E30083E0111101C082E080938B028DCF2E
:101B30008058823008F089CF8091F4019091F501AE
:101B40008C3D53E0950791F583E08A838AE289838F
:101B50004FB7F894DE01139620E03EE051E2E32F08
:101B6000F0E050935700849120FF03C082958F705E
:101B70003F5F8F708A30C0F0895C90E08D939D93B9
:101B80002F5F243161F74FBF8091E800877F8093FA
:101B9000E8006AE270E0CE01019652DB8091E80035
:101BA0008B778093E80051CF805DE7CF292F3327D3
:101BB0002330310509F44EC078F52130310509F4A0
:101BC00088C08BE590E0EDE3F2E02230310509F0CA
:101BD0003CCF2091E800277F2093E8002091F80176
:101BE0003091F9018217930708F49C0140E0211518
:101BF000310509F073C0411171C08091E80082FD88
:101C0000CDCF80918B02811549F2853039F28091D8
:101C1000E80083FFF2CFC2CF8091F6019091F701E7
:101C20002132310509F446C02232310509F00DCFC9
:101C30008330910508F009CFFC01EE0FFF1FE25A37
:101C4000FE4F0190F081E02D855A9E4FDC018C9172
:101C500090E010C09C013327823021F12330310500
:101C600068F4232BB9F4EEEFF2E0E4918E2F90E0CC
:101C7000EEEFF2E0009709F4E8CEABCF2330310568
:101C800009F0E3CEEAEAF2E0E4918E2F90E0EAEA8E
:101C9000F2E0F0CFECEEF2E0E4918E2F90E0ECEE8B
:101CA000F2E0E8CFE8ECF2E0E4918E2F90E0E8EC8F
:101CB000F2E0E0CF8330910508F0C7CEFC01EE0FD3
:101CC000FF1FEC59FE4F0190F081E02D89E090E07C
:101CD00080CF82E190E0E8E9F2E07BCF80918B0257
:101CE000811509F45BCF853009F458CF8091E80065
:101CF00083FD54CF8091E80082FD7FCF8091E80082
:101D000080FF75CF9091F3008091F200211531058D
:101D100019F08830910550F041E0089709F040E053
:101D20008091E8008E778093E80061CF44914093E2
:101D3000F1003196215031090196E8CF803809F041
:101D400084CE8091E800877F8093E8008091F00145
:101D50008093F10070CE811178CE1091F401123091
:101D600008F073CE8091E800877F8093E80010939D
:101D7000F001BFDA1115D9F084E080938B0242E0C4
:101D800061EC81E04CDB42E261EC84E048DB42E262
:101D900061EC82E044DB42E260EC83E040DB809176
:101DA0008B02843051F482E0809303014ECE809107
:101DB000E30087FDE1CF81E0E0CF81E0F5CFCF9375
:101DC000C82F811599F08CEF8C0F813A88F4ECEDD7
:101DD000F1E082EE91E02191C217B1F18E179F07D9
:101DE000D1F76C2F8AED91E0B1D8A1DCCF910895A5
:101DF00080E28C0F883048F4C77081E001C0880F02
:101E0000CA95EAF70E94F703F0CF8BE58C0F833079
:101E100030F42C2F2452330BC90148D8E7CFE8E522
:101E2000EC0FEB3148F4F0E0EE0FFF1FEE55FE4FE4
:101E30008081918163D8DACF83E38C0F8331B0F650
:101E400061E08C2F0CD9D2CF6C2F8AED91E098D81D
:101E50006EDCC7CFCF93DF93EC01805E91090897CA
:101E600020F06FE770E1209711F463E770E1CE0195
:101E70000E94E9028C2FA3DFDF91CF910895811595
:101E800061F19CEF980F913A28F4682F8AED91E068
:101E900077D84DCC90E2980F983050F4877091E04D
:101EA00001C0990F8A95EAF7892F0E94FD03F1CFAF
:101EB0009BE5980F933020F480E090E00C94560757
:101EC00098E5980F9B3118F480E090E017C893E3F1
:101ED000980F933110F460E0C2C80895CF93DF9358
:101EE000EC01CDDFCE01805E9109089720F068E813
:101EF00070E1209711F469E770E1CE010E94E902D8
:101F0000DF91CF9108950F931F93CF93DF938C01AF
:101F1000EB01A0DF209739F4C801E0DFDF91CF911A
:101F20001F910F9108958FE99FE00197F1F700C08D
:101F300000002197EFCF1F93CF93DF93182FEB0172
:101F40003EDF209731F4812F9ADFDF91CF911F91EF
:101F500008958FE99FE00197F1F700C000002197F5
:101F6000F0CF60E570E0893311F060E070E0E3CF1E
:101F7000A0E0B0E0EEEBFFE00C947E31E82FF0E063
:101F8000E354FE4FD490282F26952695269530E0D1
:101F9000F901E355FE4F0491877010E0082E02C04E
:101FA000159507950A94E2F701701127F901E35698
:101FB000FE4FE490F12C082E02C0F594E7940A94A9
:101FC000E2F7E0FAEE24FF24E0F8F901E357FE4FD0
:101FD000C491D0E002C0D595C7958A95E2F7C1704B
:101FE000DD270115110511F081EEE9DEE114F104A0
:101FF00011F086EEE4DE60E070E08D2D9CDFE114F0
:10200000F10411F086EE3BDF0115110511F081EEB0
:1020100036DFCD2B11F08CE2A4DFCDB7DEB7E7E0E1
:102020000C949A3190911604923061F48A3040F405
:10203000875F90E06AE070E00E94AA31875A91CFF2
:102040008650FDCF96EF980F963010F0805D90CFC0
:10205000895AFDCFCF93DF93EC0188818115D9F0A8
:10206000813009F03DC08981813021F48A81239635
:1020700078DFF3CF823021F48A812396A0DEEDCF82
:10208000833021F48A812396FADEE7CF843031F061
:1020900022968111E2CFDF91CF9108958A81239614
:1020A00020E030E09AE0682F6053770BAB016A3094
:1020B000710560F02115310561F3EFE9FFE031971B
:1020C000F1F700C0000021503109F4CF929FB00118
:1020D000939F700D11249A01260F371F8991E3CF2A
:1020E000219646DFBACF811519F00E94F7031FCB66
:1020F0000895811519F00E94FD0319CB08958115EB
:1021000031F090911D04892B80931D0410CB08950C
:10211000811539F0809590911D04892380931D04C9
:1021200006CB089580918C03811521F082E2F0DFC7
:1021300010928C030895CF93DF93EC014A855B8561
:102140006E857F850E943E079B81909580911D043E
:10215000892380931D048C810E94FD03E8DA86E0C8
:10216000FE0111928A95E9F7DF91CF910895CF93FF
:10217000DF93EC018D8181FD13C082608D8380919E
:102180001D049B81892B80931D048C810E94F70381
:10219000CEDA488559856E857F85CE010E943E073F
:1021A00010921104109210048D8180FD02C0CE01A6
:1021B000C2DFDF91CF910895ACE0B0E0E2EEF0E154
:1021C0000C947D31FE01319688E0DF011D928A95E5
:1021D000E9F744E051E0BE016B5F7F4F8F016A0178
:1021E000EE24E394F12C30E0D6012D916D012F3FC8
:1021F00081F0822F82958F70805E90E0DC018C915F
:1022000090E02F7002C0959587952A95E2F780FFA0
:1022100068C080E0F82A3F5FEE0C353029F7F19274
:102220004B5F5F4FE617F707D1F648E050E0B80183
:1022300083E692E00E94F7319C01892B41F088E00F
:10224000F801A3E6B2E001900D928A95E1F70091C2
:102250006C0210E00F571D4F232B09F444C081E09E
:102260008093EB010E94D1079093EA018093E901EA
:102270008091A102811509F491C07E01B9E0EB0EB5
:10228000F11C84E0F70111928A95E9F78091EC0145
:102290008A3008F04CC048E652E1B701C801CAD9FB
:1022A000811509F469C04DE052E1B701C801C2D9F6
:1022B000811509F461C01092EC0180916B0290E0ED
:1022C00044E050E0B7018F579D4F0E94F73121E065
:1022D0002093E801892B09F041C02C96E8E00C948A
:1022E00099318E2D97CF8091EB01811509F4C0CFE4
:1022F000E090E901F090EA010E94D1078E199F0950
:10230000059708F4B5CF44E050E063E672E0C801F9
:102310000E94F731892B41F084E0E3E6F2E0D80136
:1023200001900D928A95E1F71092EB01A1CFC09038
:10233000E601D090E7010E94D1078C199D09843FE6
:10234000914008F0A8CF8091E801811531F284E036
:10235000D7011D928A95E9F71092E801E0916B028E
:10236000F0E0EF57FD4F89859A85AB85BC8580836A
:102370009183A283B383B1CF8091EC018F3F39F475
:102380000E94D1079093E7018093E601DCCF8F5F35
:102390008093EC018A3008F490CFF2CFF80180816D
:1023A0009181A281B3818093910290939202A09334
:1023B0009302B093940281E992E018D8809390023E
:1023C000C0909502D0909602E0909702F09098020B
:1023D0008091E2019091E301A091E401B091E501C7
:1023E000C816D906EA06FB0609F477CFC092E201C7
:1023F000D092E301E092E401F092E5010E94EA0844
:10240000C61AD70AE80AF90AC092A302D092A40217
:10241000E092A502F092A60260CFCF92DF92EF92F7
:10242000FF921F93CF93DF9300D000D0CDB7DEB7DC
:10243000C0908C02D0908D02E0908E02F0908F02BE
:102440000E94EA086C197D098E099F0911E0643623
:1024500071058105910578F10E94F608DC01CB0138
:102460000296A11DB11D89839A83AB83BC838091A1
:1024700036019091370180579D4F20913501422FB1
:1024800050E0253010F044E050E0BE016F5F7F4F18
:102490000E94043282E090E00E940531182F8115DD
:1024A00051F00E94EA0860938C0270938D02809331
:1024B0008E0290938F02812F0F900F900F900F90AC
:1024C000DF91CF911F91FF90EF90DF90CF90089513
:1024D0008F929F92AF92BF92EF92FF921F93CF93F2
:1024E000DF9300D000D00F92CDB7DEB77B0180E044
:1024F00090E00E940531182F811509F464C0809185
:102500002801482F50E0811511F041E050E0609122
:10251000290170912A0160577D4FCE0105960E94D6
:10252000043280909D0290909E02A0909F02B090F5
:10253000A0020E94EA08681979098A099B09643691
:1025400071058105910538F481E992E00E94F60950
:102550009D818917C1F181E090E00E9405318115CC
:1025600009F43FC080913001482F50E0853010F0D1
:1025700044E050E0609131017091320160577D4F2D
:10258000CE0101960E94043281E992E00E94F60990
:102590009D81891326C00E94EA0860939D02709372
:1025A0009E0280939F029093A00289819A81AB81C1
:1025B000BC818093990290939A02A0939B02B0935E
:1025C0009C0281E00FC08091910290919202A091B3
:1025D0009302B091940289839A83AB83BC831111D7
:1025E000E4CF80E04091990250919A0260919B0261
:1025F00070919C02F70140835183628373830F9033
:102600000F900F900F900F90DF91CF911F91FF903F
:10261000EF90BF90AF909F908F9008950F931F936E
:10262000CF93DF93982F962B983020F5453010F5F7
:10263000C42FD0E0CC0FDD1F2AE0629FC00DD11D5A
:10264000112430E5839FC00DD11D1124CE01899640
:102650000E942432082F10E0102F0027CE018A9606
:102660000E9424329801282BC901DF91CF911F913C
:102670000F91089580E090E0F8CF462F672F2091CA
:10268000A9023091AA02232B81F4703F39F4403F14
:1026900061F48091A7029091A8020895982F972B3A
:1026A000983018F4453008F4B9CF80E090E00895F0
:1026B000A0E0B0E0EEE5F3E10C947E317C01009106
:1026C000D3048091D204082BC7E0D0E010E0C80109
:1026D0000C2E02C0959587950A94E2F780FD09C0FB
:1026E0002197A8F7D12C8D2DCDB7DEB7E7E00C945C
:1026F0009A31DC2EB7018C2FC0DF0E9403050197B1
:1027000079F3F1CF0F931F93CF93FC0187819085CD
:10271000009789F4858100811181811581F061150F
:1027200071F0C801C5DFC82F682FC8010E94490396
:10273000B8018C2FA2DFCF911F910F910895C8018E
:102740000E947F03C82FF4CFCF93DF93D82FC92FD8
:10275000AFDF6D2F7C2F91DF0E940305DF91CF91BA
:102760000895FC0184818115B1F0878190850097DF
:10277000A1F00E940305282F92959F709630B9F022
:1027800080F4925F9F70923030F4203FD1F058F483
:1027900081E0283E58F080E0089580819181D4DF67
:1027A000EACF9A5FEFCF81E0243FA9F7089591E047
:1027B000813F09F090E081E0283E08F080E0892B1D
:1027C000089581E00895382F292FCB01A32FB22F30
:1027D00087389105A105B10520F487589C4F0C94CA
:1027E000243280E0089585E290E00E94243281370F
:1027F00089F486E290E00E942432853C59F487E215
:1028000090E00E94243291E0843009F090E0892F1A
:102810008170089580E0FCCF80E090E00E942C322F
:10282000833E9E4F09F4DFCF80E00895AAE0B0E038
:10283000ECE1F4E10C947831C0908902D0908A02E6
:1028400081E090E090938A0280938902812C912C00
:1028500010E0540100E01AC021E030E0153020F40F
:10286000F701859195919C01472D602F812F0E9442
:10287000700B739422E0E20EF11C35E07312ECCF82
:102880000F5F85E0A80EB11C083049F0C501880F24
:10289000991FFC01EE5FFC4F7F01712CDDCF1F5FA4
:1028A000F8E28F0E911C1830A1F61A8219821C8250
:1028B0001B821E821D8218861F8288EC90E09A87F8
:1028C000898709EA12E09E012F5F3F4F79014AE0B4
:1028D00050E0B801C7010E945E32065F1F4F093FFA
:1028E00032E01307A1F78AE0F70111928A95E9F720
:1028F0004AE050E0B801C7010E945E32065F1F4FF8
:102900000934F3E01F07A1F786E0F70111928A95D9
:10291000E9F746E050E0B801C7010E945E320A5F65
:102920001F4F0937F3E01F07A1F7D0928A02C09228
:1029300089022A96EDE00C949431AAE0B0E0E3EA33
:10294000F4E10C947D31EBE0F2E080E5DF011D92D3
:102950008A95E9F7E3E2F4E088E3DF011D928A95C6
:10296000E9F78BE0C82E82E0D82E7F0109EF12E054
:10297000F701D182C0824AE050E0B801CE01019651
:102980000E94143288E0FE013196D60101900D922A
:102990008A95E1F789859A85D70113969C938E9342
:1029A0001297BAE0CB0ED11CE7E0EE0EF11C065FE9
:1029B0001F4F0934F3E01F07D9F62A96E8E00C947C
:1029C0009931A6E0B0E0E7EEF4E10C947E310CE240
:1029D00013E089E4E82E83E0F82E98E0D92E46E053
:1029E00050E0B701CE0101960E941432F8018D2DFE
:1029F00011928A95E9F7B8016C5F7F4F89819A81BE
:102A00000E942606F80191838083B8016B5F7F4F97
:102A10008B819C810E942606F801938382838D819D
:102A200086838E818783F6E0EF0EF11C085F1F4FCF
:102A300089E7E81683E0F80691F62696E7E00C941D
:102A40009A31282FCB01283070F44AE0249F90015E
:102A50001124B90167557D4F4AE050E00E941432BD
:102A600080E090E008958FEF9FEF0895AAE0B0E036
:102A7000ECE3F5E10C9483319C019755811591406D
:102A800068F4BE016F5F7F4F822FDBDF892B31F44B
:102A900089859A852A96E2E00C949F3188EC90E033
:102AA000F9CFA0E0B0E0E7E5F5E10C947E31162F18
:102AB000D72FC42FD22E8115A1F0409317040E9466
:102AC000D1079093EE018093ED01C77081E001C0C2
:102AD000880FCA95EAF707DBCDB7DEB7E7E00C94BD
:102AE0009A3190911704491333C0E090ED01F090B2
:102AF000EE010E94D1079C012E193F097901812F17
:102B00009D2FB4DFE816F90618F5D0E2DD0DCD15DE
:102B100091F0C77011E0812F01C0880FCA95EAF7C4
:102B2000E8DAD83040F48D2D877001C0110F8A95F6
:102B3000EAF7812FD8DA802F14DAD83068F62D2DF5
:102B4000277081E001C0880F2A95EAF7D2DAC4CF56
:102B5000C77081E001C0880FCA95EAF7F7CFAAE0F5
:102B6000B0E0E5EBF5E10C9473317C01DC011496E7
:102B70008C91811509F448C161E0C701C3DD8C0166
:102B8000F7018581811521F1809110049091110444
:102B90000097F1F008171907D9F0FC01FF27887F8B
:102BA0009927892B09F04BC084E0EE0FFF1F8A950F
:102BB000E1F7E057FC4F85818460858311830083B2
:102BC000CF01D5DA10921D0461E0C7019BDD8C01B5
:102BD0008091810381113AC0D70115968C9181159E
:102BE00009F4C9C00115B0E51B0708F0AFC0011515
:102BF000E0E21E0708F00CC10115F7E01F0731F1F4
:102C000008F5C801805E9109089700F130911B0416
:102C100080911D0420911A0499E0F701ADE6B3E01C
:102C200001900D929A95E1F7109375030093740348
:102C300010927703832B822B80936C0307C0E0E014
:102C4000F0E0B9CF01153FE0130701F7F7018581E7
:102C50008111DBC1011527E5120708F4E6C2011551
:102C600038E5130710F00C94B91F680147E5D41A32
:102C700062E873E08C2DE5DE892B31F5C601F4E0C6
:102C8000880F991FFA95E1F7FC01E057FC4F22816C
:102C9000213009F09AC22091820330918303232BC3
:102CA00099F02091840330918503232B69F02091C2
:102CB0008603309187034091880350918903242B28
:102CC000352B232B09F48BC280918C03811509F4D9
:102CD000B9C3C0901B04D0901A040E94D107885732
:102CE0009C4E90938E0380938D03D70115968C9103
:102CF000811509F4A7C38D2D8C298D7981115EC3AF
:102D00000115B0E51B0708F0E6C20115E0E41E0757
:102D100008F081C3063E110509F40BC3C8019052A7
:102D20008115904208F07EC3D70116968C918031B0
:102D300008F43BC3C801992710921D048D329105F8
:102D400009F0E2C282E080931D0470C3003E42E5B8
:102D5000140750F4003652E5150708F077CFC80184
:102D600092558034910551CF980127573C47253023
:102D7000310508F04BCF0937BCE71B0709F04DC000
:102D80002091740330917503232B69F1811599F01B
:102D900081E00E94180780916C03B1D989E0EDE6CB
:102DA000F3E0A3E2B3E001900D928A95E1F7809100
:102DB00077038093220386E0F701A3E2B3E001905A
:102DC0000D928A95E1F7809122038093810383E23B
:102DD00093E0C5DE10928103F7018581811103C064
:102DE00080916C0395D980911E048770811561F0E4
:102DF000D70115968C91811539F08091D50482FF09
:102E000003C082E00E94DC032A96E2E10C948F3139
:102E1000D70116968C918031F8CE0A37FCE71F0750
:102E200009F014CF811509F4C5C0A0907403B090C7
:102E3000750320916C032D832983BE016F5F7F4F43
:102E4000C5010E9426062C0139813A87BCE2CB2EAF
:102E5000B3E0DB2E01E010E022242A94D60117967D
:102E60003C90179733FE53C06D907C90119712964B
:102E70008D909C90139746145704B9F41496BC9106
:102E8000B987232DF60146816B2F8A850E94400663
:102E9000811559F089850E941503281634F4D6014E
:102EA00015969C918401192B282E48145904C9F4B5
:102EB00031FE17C0F601F581F987232DD60116964C
:102EC0004C916F2F8A850E944006811551F08985AB
:102ED0000E94150328162CF4F60194818301192B06
:102EE000282E30FE14C0FFEF2F1211C00130110543
:102EF00071F4232DD60116964C9160E08A850E94CC
:102F00004006811521F0F60185818401182BF8E037
:102F1000CF0ED11C2CE633E02C153D0509F09ECFD9
:102F200001301105E1F58D8182958F703D81832BF4
:102F30008F7011E0303108F410E01295107F182BDB
:102F4000A11440E2B40620F5A11451E0B50608F042
:102F500055C00A2D812F8D704A2D811509F451C05D
:102F60006AE08CE895E00E942907282F30E02115BF
:102F7000310551F4402F6EE186E695E00E94290765
:102F8000282F30E0811549F0F901F12B8F0107C09E
:102F9000C50190528115904390F100E010E087E068
:102FA000E8E7F3E0DF011D928A95E9F710938003CB
:102FB00000937F0380917F0390918003892B09F414
:102FC00012CFF7018581811539F08FEF0E94180724
:102FD000809177038093760386E0F701A8E7B3E05A
:102FE00001900D928A95E1F7809176038093810399
:102FF00088E793E0B4DD10928103F5CE1B29BB2452
:10300000A8CF68E084E895E0AECFC8019757803834
:10301000910508F0EFC0003108F0E5CE66E870E0F9
:1030200080E090E0D0DB8111DECE812C912C540128
:10303000011144C004E0AE014F5F5F4F6A01D60149
:10304000E02F1D92EA95E9F724013501FFEF4F1AB1
:103050005F0A6F0A7F0AC501B401B5DB8983811558
:1030600009F4C1CE813009F0ACC0A50194012E5FF6
:103070003F4F4F4F5F4F2D833E834F835887C30190
:10308000B201A1DB182F8A83811509F4ACCE8FEF32
:10309000810F833058F56D817E818F81988593DB18
:1030A0008B83811519F0C6010E942A102401350175
:1030B00033E0430E511C611C711C46C0F7E88F16AB
:1030C0009104A104B10409F48ECEC501B4017BDBE7
:1030D0002FEF821A920AA20AB20A8111EFCF015091
:1030E000A7CF4D805E806F8078842EC08BEF810FDC
:1030F000833098F52401350143E0440E511C611CD6
:10310000711C6D817E818F8198855DDB8B8381153C
:10311000D9F0C301B20157DB8C83811571F08B812B
:103120009C8181305FEF950710F0982F882716302B
:1031300071F0173079F00E94D2252401350154E056
:10314000450E511C611C711C5301420178CF0E9435
:103150009025F3CF0E94B125F0CF143009F0C1CFF4
:103160006D817E818F8198852EDB182F240135019A
:1031700084E0480E511C611C711CC501B4016D5FD7
:103180007F4F8F4F9F4F1FDB111509F42CCE8115F8
:1031900009F429CE8150990B4FEF489F9001499F28
:1031A000300D1124A12FA150BB0B2A0F3B1F215022
:1031B000310950F2EFE9FFE03197F1F700C000006C
:1031C000F6CFC6010E942A10BFCF223009F07CCD75
:1031D0002091860330918703232B09F475CDFC01E0
:1031E000EB56FC4F20812E7F208380579C4F0E94FE
:1031F000B7106ACD03375CE71507B9F480918C03EB
:10320000811519F00E949210EECD10921B040E94BD
:1032100005040E94D10788579C4E90938E0380939B
:103220008D0381E080938C03DECD023A82E518079E
:10323000C1F158F4C80190528115904220F1013E2D
:10324000110579F1053E110503C0023BB2E51B07EC
:1032500009F03ACD25EE30E02770332781E090E089
:1032600001C0880F2A95EAF720918F0330918C03D3
:103270003115F9F0D70115963C913115A9F0282B9D
:1032800020938F03B0CDF7018681803108F01CCDEB
:10329000812F99278F7199278230910511F04297DC
:1032A000D7CF21EE30E0D8CF8095822380938F0353
:1032B0009ACD322F3823311509F406CD982F9095E9
:1032C000922390938F030E94FD03F701858181155E
:1032D00009F489CDF9CC003EB2E51B0708F058C0CF
:1032E000003CE2E51E0728F5003AF2E51F07E8F486
:1032F000003622E51207E8F4C801925580349105A2
:10330000C0F010921D04C8018E32910508F0E1C092
:103310008832910508F088C08E31910508F086C08A
:1033200004974A9708F40ECD49C0043B32E51307D1
:1033300041F7D7011596DC90D11409F4ACC117FF01
:10334000AAC12801E89457F8612C712C0E94430708
:103350008093150490911604913029F481FF03C0E5
:1033600089E30E94B10F80911B0480931404109292
:103370001B0410921D0480911604823009F41BC1B5
:1033800008F0E0C0811110C182EE0E94DF0EE0C0A3
:1033900009374CE7140728F407375CE7150748F6A8
:1033A000B0CF0B378CE71807C3CF812F8F718431D3
:1033B00009F4BFCF863149F410921D040E94921087
:1033C00080918F030E94F7033DC00E94921080916C
:1033D0008F030E94F703F7018581811509F4A9CFB6
:1033E0000533FCE71F0709F4A9C008F096C00333B2
:1033F0003CE7130709F49EC004334CE7140709F4B3
:103400009BC002335CE7150709F093CF10921604B6
:103410000E946A0B8ECFD70116968C91803108F0EE
:1034200089CCD9CFC80188CC8A9741F680918F0387
:10343000811531F080911D0492E0892780931D044D
:103440000E94970BC80197558115914020F65801AD
:10345000F8EFAF22BB24A114B10409F0C4CCF801E9
:10346000FF2774E0EE0FFF1F7A95E1F79F012057C9
:103470003C4F6901D70115968C91EB56FC4F90811A
:1034800080FB90F99083811559F10E94D1079093A8
:10349000130480931204F60182818F5F82838091EE
:1034A0001D0490911B04892B838380911A048483CB
:1034B0004681578166857785C6010E943E07D60101
:1034C00015968C9181FF5801B0921104A0921004BE
:1034D00082CF8C34910509F4A9CF8D329240A5CFCB
:1034E000F9014485558566857785C9010E943E07A7
:1034F000D60115968C9181FF6ECFC6010E949B105C
:1035000080911004909111040817190709F063CFF6
:1035100010921104109210045ECF06338CE7180746
:1035200079F085E007339CE7190709F002CF809313
:1035300016046ECF81E0FBCF82E0F9CF83E0F7CFB6
:1035400084E0F5CF843009F44AC0853009F44CC0DA
:103550008FE39CE90197F1F700C00000C0901604CA
:103560005CE1852E912C67E0A62EB12CD301C2011F
:10357000082C04C0B695A795979587950A94D2F71D
:10358000E82FEF703E2ED11451F0F4E0CF12D2C4E8
:103590002AE0E21708F4CEC480E00E941210832DC6
:1035A0000E941210D12CCDC460E070E088E193E05D
:1035B0000E94830FCDCF8091150480FD03C083E569
:1035C0000E94B10F82EE0E94DF0EEFE3FCE931971B
:1035D000F1F700C0000087E50E94B10FB9CF86EE79
:1035E0000E94B10F88E1F8CF60E070E08BE191E0DC
:1035F0000E94830F60E070E085E290E00E94830FFC
:1036000060E070E088E290E0D3CF8430D9F185307B
:10361000D9F18091140480931B04D70115969C91D5
:10362000911509F4AAC41092170498013057233257
:10363000310508F0B2C484E090E00E942C329093EF
:10364000D5048093D404F801E150F047E232F1054B
:1036500008F058C0EC56FD4C0C94BD318CE20E9431
:10366000B10F8091150481FFD4CF89E30E94B10F7F
:10367000D0CF82EE0E943F0F8091150480FDC9CF0C
:1036800083E5F4CF88E2F2CF60E070E088E290E07A
:103690000E94830FBECFF801E851FC47E730F105E7
:1036A00008F0BBCFEA54FD4C0C94BD3106E221EE8C
:1036B00041EE6AE17CE78D2DF4D995CB07E225EE4A
:1036C00045EE6BE17CE7F7CF06E221EE40EE68E1E4
:1036D0007CE7F1CF07E225EE44EE69E17CE7EBCF32
:1036E00006E221EE42EE6CE17CE7E5CF07E225EE53
:1036F00046EE6DE17CE7DFCF08E221E045EE6EE1CA
:103700007CE7D9CF8091D40481608093D404609108
:10371000D4047091D50484E090E00E945A320E9453
:10372000E40B61CB8091D50488608093D504EFCF02
:103730008091D4048260E9CF8091D4048460E5CF85
:103740008091D4048860E1CF8091D5048160EDCF71
:103750008091D5048260E9CF8091D4048061D5CF77
:103760008091D4048062D1CF8091D4048064CDCF85
:103770000E94E40B8091D4048068C7CF8091D40468
:103780008C60C3CF8091D5048360CFCF8091D40467
:103790008E7FBBCF8091D504877FC7CF8091D40423
:1037A0008D7FB3CF8091D4048B7FAFCF8091D40431
:1037B000877FABCF8091D5048E7FB7CF8091D50422
:1037C0008D7FB3CF8091D4048F7E9FCF8091D4041E
:1037D0008F7D9BCF8091D4048F7B97CF0E94E40B89
:1037E0008091D4048F7791CF8091D404837F8DCF43
:1037F0008091D5048C7F99CF8091D404992782FF42
:10380000939590FB82F990FB83F97FCF8091D5044B
:10381000982F909590FB80F990FB81F986CF90913D
:10382000D404892F8F7B96FF80646FCF0E94E40BB6
:103830009091D404892F97FB87F9805866CF61E077
:103840008EE090E00E94403262CF60E0F9CF90912C
:10385000D404892F8F7E94FF806157CF9091D40438
:10386000892F8E7F90FF816050CF9091D504892F52
:10387000877F93FF886059CF0737BCE71B07F9F0B4
:103880000837ECE71E0731F19801205E32452032FF
:10389000310528F5911123C00F7181E090E09C0162
:1038A00002C0220F331F0A95E2F78901622F83E0DD
:1038B00090E00E944032802F0E942B0394CA81E046
:1038C000911551F00E94310343E062E081E00E94D3
:1038D000B30389CA82E0F4CF0E943B03F5CF409145
:1038E00019048091D304282F30E02095309570E0A2
:1038F00024233723232B19F04823409319040B3733
:103900003CE7130741F4911509F46DCA0E941803AE
:103910000E949E0668CA003442E5140708F055C0AC
:10392000003252E5150708F057C0011580E5180769
:1039300050F50115A0E41A0708F064C0911509F4C8
:1039400079C00A35FCE71F0709F4CDC008F0B2C002
:1039500001303CE7130709F4C4C003304CE71407F7
:1039600009F4B9C001151C4709F064C00E94E40BBA
:10397000AFEFB4E3ECE0A150B040E040E1F700C0AD
:1039800000000E940E099801305521153240B0F612
:10399000980145E0369527954A95E1F7822F8F707B
:1039A0002091190430E041E050E0082E02C0440F9D
:1039B000551F0A94E2F724233523232B09F4BECFA5
:1039C0009111A6CF10921B04FEC29801205C3245D3
:1039D0002032310508F0B2CF802F8F712091190469
:1039E00030E041E050E0082E02C0440F551F0A9419
:1039F000E2F724233523232B09F4A0CF911509F4F2
:103A0000F2C986CFF7018681803108F097CF9111F6
:103A100011C0212F2F7081E090E002C0880F991F04
:103A20002A95E2F72091190430E082239323892B11
:103A300009F0D9C9F70187819085009709F457C02B
:103A40000E9403058C01F701B580A680A2942FE0A7
:103A5000A22280911E048770811501F1CB2CB11434
:103A6000F1F0812F807F803461F080E2800F883018
:103A7000A8F0812F807E803221F4023078F0A114EA
:103A800069F08091D50482FF09C082E00E94DC03C6
:103A900080911E048770CC24C3948111C12CE12F26
:103AA000E295EF70103C08F094C0F0E0E354FD4C58
:103AB0000C94BD310B358CE71807B9F08091D50413
:103AC000002482FF0394802D0C351C4709F0B2CFEF
:103AD0000E94540BAFCF6FEF7FEF80E090E00E9429
:103AE0005A320E94070C81E0F3CF80E0F1CF85814C
:103AF000C080D180811569F0C6010E945813182F2B
:103B0000682FC6010E944903B601812F0E943D1310
:103B100097CFC6010E947F03182FF6CFF12FFF70B9
:103B2000DF2E103118F0D29490EFD922B114A9F001
:103B3000D11459F080E2800F883010F0011107C0D5
:103B40008D2D0E94F7030E94970B802F40C080911B
:103B50001D048D2980931D04F6CF802F0E943F0FF6
:103B6000D114B9F180E2800F883010F0011104C047
:103B70008D2D0E94FD0306C0D09480911D048D21DF
:103B800080931D040E94970B24C0212F2F70D22EEA
:103B9000107F103219F0D29480EFD822011549F02D
:103BA000013009F483C0B11409F48FC0A114A9F144
:103BB000CCCF8091D50482FD2CC0B11421F1D11459
:103BC00029F08D2D0E94F7030E94970B80E00E9440
:103BD000DF0EC11409F4D9C080911E0480FDD5C048
:103BE000D70115961C928695869586950E9431037D
:103BF000C7010E94AF1580911E0486958695869513
:103C00000E943B03C2C080E00E943F0FD11409F321
:103C1000AFCFB11469F1A11004C08D2D0E947310B3
:103C2000D8CF31E0A31210C010911A048D2D81233A
:103C3000D81679F20E94D107909322048093210430
:103C40001D2910931A04C5CF45E0A412C2CF8D2DB3
:103C50000E9473108D2D0E94F10780911C049D2DF0
:103C60009823D91609F4B5CF8D2980931C04B1CFC0
:103C7000A11012C08D2D0E9479108D2D0E94F10788
:103C800080911C049D2D9823911509F4A2CFD09406
:103C9000D822D0921C049DCF51E0A5129ACF8091DA
:103CA0001B048D21811509F494CFE4CFB11429F0C0
:103CB00086E0A81608F08DCFB0CF95E0A91608F0E1
:103CC00088CF8D2D0E94791084CFA114D1F30933B0
:103CD00049F4AFEFB7EEE3E0A150B040E040E1F7C8
:103CE00000C00000802F0E943F0F73CF812F869568
:103CF00086958370811561F0813009F06ACFC80123
:103D00009370B11002C080E090E00E947E0761CF06
:103D1000C8019370B11002C080E090E00E94560785
:103D200058CF6B2D802F0E942F0853CF812F837087
:103D3000811138C0B11027C0402F42954695477079
:103D4000440F440F802F8F70042E01C0880F0A94F7
:103D5000EAF7202F207104FF07C02FE030E001C0F8
:103D6000220F4A95EAF72095169516951370123092
:103D7000A1F0133081F03091D204113059F0822B30
:103D800083230E942B030E94430760E0C7010E9427
:103D900082133AC8832B822BF4CF822B9091D204CA
:103DA0008927EFCFB11451F110FFEDCF402F42958D
:103DB00046954770440F440F802F8F70042E01C02A
:103DC000880F0A94EAF7202F207104FF07C02FE024
:103DD00030E001C0220F4A95EAF720951695169516
:103DE0001370123089F0133069F03091D304113020
:103DF00041F0822B83230E942E03C5CF823018F21C
:103E0000D5CF832B822BF7CF822B9091D304892798
:103E1000F2CF1F70B11439F0812F0E943103802F2F
:103E20000E947310B0CF802F0E947910812F0E94C2
:103E30003B03A9CF023F71F170F4003FC9F0013F8D
:103E400091F0B11409F465C0A11409F45FC0802F8A
:103E50000E94DF0E98CF033F21F1043F91F780913C
:103E6000D50482FD2AC0812F8F71B11401F316C0D1
:103E7000B11469F0F5E0AF1608F085CF1F7181E04D
:103E800090E0012E01C0880F0A94EAF7BECF26E029
:103E9000A216F2CF812F8F71B110C9CF0E943103CA
:103EA00072CF80E0B11409F4A6CF1F7181E0012E1A
:103EB00001C0880F0A94EAF79ECFB114C1F0809137
:103EC0001E048770843049F410921E04109220045E
:103ED00010921F04812F8F71AACF35E063E0A316E3
:103EE00008F051CF812F8F710E94DD074CCF45E044
:103EF000A41640F010921E041092200410921F0489
:103F000064E0F0CF81E00E94DC033DCF812F8F7110
:103F1000C5CFA114F9F2093349F45FEF87EE93E0BE
:103F2000515080409040E1F700C00000802F0E9477
:103F30003F0F29CF311033CB34E0A316B1040CF47A
:103F40002ECB41E0A41AB10854E0851A91088FEFF6
:103F5000A816B80609F00ACB80911604823009F43D
:103F600088CB08F052CB811179CB82EE0E943F0FB3
:103F700050CB0337BCE71B07ABC90631FCE71F0773
:103F800009F07ACC8091180465E3811101C069E2DF
:103F90008AED91E00E94C00716C006312CE7120797
:103FA00009F06ACC80911B048A7A91E0811101C0EA
:103FB00090E09093180465E3811101C069E28AEDF5
:103FC00091E00E94A6070E94970B0C94F316A0E0C4
:103FD000B0E0EDEEFFE10C947E318091070380317B
:103FE00008F049C080910603811509F444C0C091CE
:103FF000B80289E0D82E8091B7028C17E1F1EC2E3F
:10400000F12CDC9EE0011124FE01E754FD4F848178
:104010008115B1F1918180910203981331C0908193
:104020008091010398132CC08581811129C00281E0
:1040300013818091030390910403081B190B60E026
:1040400081E093E00E9482130E9436150817190739
:10405000B8F4809107038F70806180930703C15487
:10406000DD4F88818F708061888381E093E00E94BA
:10407000AF150E94D203CDB7DEB7E7E00C949A31BA
:10408000E7012196C770B7CFAFE0B0E0EAE4F0E215
:104090000C9476318C0186E0F801DE011A960190CD
:1040A0000D928A95E1F7F801F580E48081E0882E91
:1040B00083E0982E80910503811117C0E11491F0DF
:1040C000F11409F480C1C8010E94B113811509F4EB
:1040D0007AC189E0F801A1E0B3E001900D928A95E0
:1040E000E1F775DFFF24F3946AC0A280B380D0901B
:1040F000060380910303909104033501681A790A3D
:10410000D11409F411C1C080518060E081E093E0D6
:104110000E9482130E9436156816790608F0B6C010
:10412000E11401F380910203F8019181E09007030B
:10413000F0E1EF1608F064C0981320C090910103DD
:10414000F801808198131AC0209108033091090367
:10415000878190852817390789F4F1104BC08E2D7F
:104160008F7080618093070381E093E00E94AF1518
:1041700080910703F8018683F12C21C0F1103AC029
:1041800040E0652D8C2D0E94990A40E0652D8C2D14
:104190000E94990AF82E8111EFCF8A859B850E9493
:1041A000A413292F22952F70903470F49F70223021
:1041B000A0F09115B1F0F8019681903190F48F2D17
:1041C0002F96EFE00C9492312A5F2F70223068F026
:1041D000C8010E94AF15FD2CF2CF911511F0811589
:1041E00071F3805E883058F3F3CF803F40F3815FF6
:1041F0008330F9CF80910703816080930703BCCFA0
:1042000098131EC090910103F8018081981318C083
:104210002091080330910903878190852817390779
:1042200079F4F1100DC0E682C8010E94AF1589E053
:10423000F801A1E0B3E001900D928A95E1F752CF29
:10424000C8010E94B113811509F4BDC0F11409F42D
:10425000BAC080910703803208F43BCF80910103FC
:10426000909102039A838983BC82AB82809105037B
:104270008D831E82EF8280910803909109039987B4
:104280008887CE0101960E94AF1523CFD0900703F7
:10429000F0E1DF1650F481E093E00E94AF1589E071
:1042A000F40111928A95E9F767CFE11409F41ACF66
:1042B00090910203F801818198131AC09091010333
:1042C0008081981315C020910803309109038781DC
:1042D00090852817390761F4F1100AC0D682C80109
:1042E0000E94AF1589E0F40111928A95E9F7FACEA0
:1042F000C8010E94B113811509F465C0F11409F4D5
:1043000062C080910703803208F4E3CE80910103FC
:10431000909102039A838983BC82AB8280910503CA
:104320008D831E82DF82A7CF60E081E093E00E9450
:1043300082130E9436156816790608F0B0CFE11492
:1043400009F4D0CEF11409F43EC090910203F801B3
:10435000818198132EC0909101038081981329C008
:104360002091080330910903878190852817390728
:1043700001F58091030390910403A81AB90AF8EC9F
:10438000AF16B10408F053CF8091070380FD4FCFE3
:10439000803108F44CCFF8018683982F907F903FAE
:1043A00009F442CF982F907F905F8F70892B86837E
:1043B0003BCFC8010E94B11381118BCE80910703BE
:1043C000816080930703C8010E94AF158BCEA2E1E4
:1043D000B0E0EDEEF1E20C9481310A871B872C8767
:1043E0003D874E875F87688B798B8A8BCE010A96D3
:1043F0004BDE811128C02091B7023091B80289E0CC
:10440000FE013A96DE01119601900D928A95E1F730
:104410008E858115C1F0822F90E0019687709927D3
:1044200038171906D9F099E0929FD0011124A754AA
:10443000BD4FFE01319601900D929A95E1F7809360
:10444000B7020E94D20319E08091B8029091B7029E
:10445000891312C06296E4E00C949D310E94E40B33
:104460001092B7021092B80289E0E1E0F3E0DF01B8
:104470001D928A95E9F7E7CF189FC0011124875450
:104480009D4F02DE811531F38091B80290E00196D4
:10449000877099278093B802D7CFEF92FF920F933E
:1044A0001F93CF93DF938091CF04E0910A02CDE078
:1044B000811130C0CDB7DEB7E6E00C949B31D1E07E
:1044C000DE0FD0930A02EE2EF12CCE9FF0011124C4
:1044D000E959FB4F84818115E1F087819085892B13
:1044E00021F481859285019651F400811181228108
:1044F00033814481558166817781808568DFCE9DD7
:10450000F001CF9DF00D1124E959FB4F1482109258
:104510001D04ED2F8091CF04E81788F21092CF048C
:1045200010920A02C7CFA4E0B0E0E9E9F2E20C94ED
:10453000743120916604298397E0992E01E010E000
:104540002DE0322E34E0532E88248394809165042C
:104550009981891307C0A1DF0E9461062496E1E1D9
:104560000C9490319981892F90E09C838B83FC017E
:10457000EE0FFF1FE55AFB4F80819181989ED0017D
:10458000999EB00D1124FD01ED5DFB4FFA83E98387
:10459000248121115BC06090CF04E7E6F4E060E085
:1045A00070E0712C661508F04FC0A384B484A98113
:1045B000BA81CD90DC902FEF3FEF412C442D50E09D
:1045C0007601E40CF11CE40CF11CD701ED90FC9099
:1045D000E114F10439F0AE14BF0409F0A9014394C9
:1045E0009A01ECCF2F3F3207D1F1D80102C0AA0FB8
:1045F000BB1F2A95E2F77A2A9801042C02C0220FE9
:10460000331F0A94E2F7A9014150510974161506A7
:1046100029F5369EF001379EF00D1124E959FB4F24
:10462000989ED001999EB00D1124AD5DBB4F12969E
:104630002D913C91139730872783548210821182E9
:104640009287818715968C920E9472068B819C813D
:1046500001969A8389838370898378CF14826F5FF0
:104660007F4F3D969FCF1092D1041092D0041092AC
:104670003D0180916504809366040E9461060DCF20
:10468000ACE1B0E0E6E4F3E20C9473314B8B5C8B6D
:104690006D8B7E8B8F8BB92E988FA92E91111092D6
:1046A0001D04188A198A1A8A86E0FE017396DE01B3
:1046B0001A9601900D928A95E1F75F888091D50452
:1046C00082FF1FC00E94D10720911F043091200457
:1046D000821B930B8838934138F080911E0482FD31
:1046E00003C082E00E94DC030E94D10720912104D4
:1046F00030912204821B930B8838934110F00E9462
:1047000005045114D9F05E86BF8661E0CE010A9699
:104710000E94821361E0CE010A960E94821361E03A
:10472000CE010A960E9482134C0180356CE79607F1
:1047300091F4A11419F181E080933D015E86BF865A
:104740000A851B852C853D85452D5B2D68897989DA
:104750008A893DDECDC081359C4721F4A11471F0DA
:1047600082DFECCF82E588168CE7980639F4A11435
:1047700029F080913D018111F3CFDDCF43E2E42E9A
:1047800044E0F42E412C612C712CD7016D917C9169
:10479000CC24CA94DD24DA9480E0282F30E0FB0199
:1047A000E80FF11DE80FF11D4081518141155105C0
:1047B00039F08416950609F096018F5F6901EDCFF7
:1047C00010E0BFEFCB16DB0609F44EC0F7014481C1
:1047D00010913D01411110E0D70115963C901597BD
:1047E00016969C911697A11409F405C1111509F4A8
:1047F00002C1311017C021E030E00C2C01C0220FA3
:104800000A94EAF7922B16969C93209163043091B8
:1048100064042233310530F422E330E03093640441
:1048200020936304E1E0F0E002C0EE0FFF1F8A95E1
:10483000E2F7CF010197D70116962C912817190698
:1048400099F4C090D004D090D104C114D10409F4DB
:1048500053C00E94D1078C199D09C39708F44CC01E
:1048600081E0F701848311E0412ABFEF6B1A7B0AD4
:10487000E7E0EE0EF11CF8E06F16710409F085CF49
:10488000A11409F417C1411409F414C10E94D107FD
:104890009093D1048093D0048091CF04883040F568
:1048A00091E0980F9093CF0499E0FE013A96DE01D3
:1048B000119601900D929A95E1F75D82BE822DE0EE
:1048C000829FC001112489599B4F29E0FE01319636
:1048D000DC0101900D922A95E1F72FEF3FEFDC010B
:1048E0001A963C932E9319971C969C928E921B9726
:1048F0006C96E2E10C948F312091660480916504FE
:10490000922FE0E0F0E001E0281709F448C0422FC0
:1049100050E0FA01EE0FFF1FE55AFB4F2080318077
:1049200037E0329DF001339DF00D1124ED5DFB4F1A
:10493000608171817C8F6B8FB0E030E0A0E0EB8D07
:10494000FC8DEA0FF11DEA0FF11DC080D180C1146A
:10495000D104E1F0F7010190F081E02DFA8FE98FA9
:1049600030E007C0E1E0C616D70609F0E0E0BE2B54
:104970003F5FE98DFA8DE30FF11DE30FF11D6081BB
:1049800071816115710571F7AF5FD9CFB11581F1F3
:104990003A17C8F4E1E0D7011496EC93F70190932D
:1049A0006604EE15FF0509F45FCF90E0FC01EE0F01
:1049B000FF1FE55AFB4F7182608201968370992731
:1049C0008093650451CF37E0329DF001339DF00DA7
:1049D0001124ED5DFB4F0483EE15FF05F9F2291359
:1049E00002C09F5F93709A012F5F3F4F23708CCF5F
:1049F000E0E0F0E0F8CF292F30E0311024C061E092
:104A000070E002C0660F771F8A95E2F7CB0101972D
:104A10002817390791F010E0E1E0F0E002C0EE0F56
:104A2000FF1FCA94E2F76F01C094D70116968C91CC
:104A300016978C2116968C9317CF411569F3C301F5
:104A40000E947206E8CFA9010C2C02C0559547952B
:104A50000A94E2F7C901019782239323892B39F540
:104A600040FF25C0D70112968D919C91892BD1F0E2
:104A700087E0FE013196DF011D928A95E9F70E94D9
:104A8000D1079C018B839C8384E08D83F701928105
:104A90008381792F9887898709811A8144E05E8113
:104AA0006F8195DCD70115961C92132DB5CF142F6D
:104AB0001170B2CF9091660480916504981731F01F
:104AC00032DDB1E04B1609F413CF38CEE6DC10929C
:104AD000D1041092D0040E946106F3CFA6E0B0E0AA
:104AE000E4E7F5E20C9481310E94D1078C018091BA
:104AF000AB029091AC028017910771F019821A8273
:104B00000E94D107BC0149815A8180E090E0B8DD64
:104B10001093AC020093AB022696E4E00C949D3116
:104B2000A6E0B0E0E6E9F5E20C9483319093A802A8
:104B30008093A702811520E2920730F40E942A0F89
:104B40002696E2E00C949F3180EF89838A830E944D
:104B5000D1078160BC0149815A8181E091E090DDFB
:104B6000EFCFA6E0B0E0E7EBF5E20C948331909351
:104B7000A8028093A702811520E2920730F40E94D8
:104B80006E0F2696E2E00C949F3180EF89838A8332
:104B90000E94D1078160BC0149815A8181E090E087
:104BA0006FDDEFCFCF93DF93D82FC92FB9DF8D2FD4
:104BB0009C2FD7DFDF91CF9108950F931F93CF9351
:104BC000DF938C01862F62E873E00E942115892B08
:104BD00091F4C0918203D0918303209761F0F80192
:104BE0008281833039F4CE01DDDFCE01DBDFCE01FF
:104BF000D9DF01C0E0F7DF91CF911F910F910895A8
:104C00000F931F93CF93DF938C01EB0162E873E066
:104C10008C2F0E942115892B09F057C0FE01FF2718
:104C2000D80112968C911297E55AFD4F8130A9F464
:104C300015968C9182FD4EC080FF4CC082E080832F
:104C400080918403909185030097B9F48091820349
:104C5000909183030097C9F110C08230A1F5159699
:104C60008C9182FD26C080FD0AC083E08083809104
:104C70008603909187030097F1F052DF26C084E00D
:104C8000808380918803909189030097B1F7809188
:104C9000820390918303009701F184DF8091840364
:104CA00090918503009749F7809182039091830347
:104CB000E4CF85E080838091820390918303009705
:104CC00021F070DFF1CF86E08083DF91CF911F91DB
:104CD0000F91089581E08083B9CF809184039091F2
:104CE0008503B8CF0F931F93CF93DF938C01EB0114
:104CF00062E873E08C2F0E942115892B71F4DD2767
:104D0000C55ADD4F8881F801128218828330E9F09C
:104D100048F4813059F0823081F0DF91CF911F91BA
:104D20000F9108958430B1F08530B9F780918203F6
:104D300090918303009789F306C08091840390913A
:104D40008503009799F30DDFE8CF8091860390915A
:104D50008703F7CF8091880390918903009799F793
:104D60002091820330918303809184039091850385
:104D700021153105F9F2009731F7C901E4CFA0E11F
:104D8000B0E0E5ECF6E20C947531FE01319680E17D
:104D9000DF011D928A95E9F709E010E099E7A92E55
:104DA00093E0B92E27E8422E512C612C712C4F0133
:104DB00073016201B1E14B165104610471041CF0EE
:104DC00080E1C82ED12CA601B501C4010E94313268
:104DD000AC0CBD1C0D2C000CEE08FF084C185D0837
:104DE0006E087F080150104019F76096E0E10C94BE
:104DF00091316FEF85E290E00E9440326FEF86E2E2
:104E000090E00E9440326FEF87E290E00E944032D3
:104E100060E088E290E00E9440320E941614AFDF0A
:104E200061E785E290E00E94403265EC86E290E026
:104E30000E94403264E087E290E00C94403263EEDE
:104E40007EEF80E090E00E945A3260E082E090E0E5
:104E50000E94403281E08093D20461E083E090E0E0
:104E60000E94403260E074E184E090E00E945A3297
:104E700060E08CE090E00E944032BBDF40E050E018
:104E8000BA018FE090E00E94523240E050E0BA0157
:104E900083E190E00C945232CDB7DEB7AC970FB6F9
:104EA000F894DEBF0FBECDBF85B7806885BF85B7DC
:104EB000806885BF84B7877F84BF0FB6F894A895B4
:104EC00080916000886180936000109260000FBE46
:104ED00080E890E00FB6F8948093610090936100B1
:104EE0000FBE81E0809303018FEF95E09093D9018D
:104EF0008093D8010E940E060E949D140E94E11426
:104F00000E94C9090E943F0A8091E2008460809358
:104F1000E200789480918B02811599F08091E900EC
:104F20001091EC008F70179511271795182B109280
:104F3000E9008091E80083FD0E941C0C1F70109313
:104F4000E90082E084BD93E095BD9AEF97BD809320
:104F50006E001092A3021092A4021092A502109269
:104F6000A6020E94F313811101C043DF8091D80093
:104F700080618093D8002AE12A95F1F700C08091E2
:104F8000D900182F117080FD04C00E94C909109229
:104F90008B021093A1020E940C14811101C04FDFFB
:104FA0008EE090E00E94243291E0811101C090E0F7
:104FB0009093A202909318018091A10281110E9406
:104FC000203080911801811112C084E1EEE3F1E0FC
:104FD000DE01119601900D928A95E1F784E1FE01C0
:104FE0003196A4E0B1E001900D928A95E1F78091AD
:104FF000180191E08927880F880F80936C0294E054
:10500000981B90936B0224E031E068E171E001E0CD
:1050100010E0D90140E050E08D918F3FA1F0E82FE2
:10502000E295EF70F0E0F1A08F70680102C0CC0C47
:10503000DD1C8A95E2F7C6019C2D90959F2191A3D6
:1050400092A1892B82A34F5F5F4F4530510521F715
:105050002B5F3F4F62177307E1F688E0E1E8F2E06B
:10506000DF01C82E1D92CA94E9F7E3E6F2E0DF0102
:105070001D928A95E9F70E940C14811101C0DFDEB0
:1050800082E090E00E94243280936F0284E090E0FE
:105090000E942C329093D5048093D4040E94DC109B
:1050A000BFEFE6E7F1E0B150E040F040E1F700C0CB
:1050B00000000E94DC108091A20291E08927880FF5
:1050C000880FE82FF0E0EF57FD4F208130E041E0FE
:1050D00050E06A0102C0CC0CDD1C8A95E2F7C601E3
:1050E00082239323892B41F06FEF7FEF80E090E0E4
:1050F0000E945A320E940E0983E090E00E942432FE
:105100000E942B038CE090E00E94243280931604CE
:105110008091A102811101C096D789E191E090931D
:10512000AE028093AD0280918B02853049F480916C
:105130008B02853009F452C00E94E40B0E944307A1
:105140000E94DC1000E712E061E8E62E62E0F62E35
:10515000D701F80191918D9158E7C52E52E0D52ED7
:10516000CE16DF0609F46FC09817A1F38090A10254
:10517000D12CD701CD907D01F80191908F019C1425
:1051800031F19C24B12CAA24A394892D8A21811564
:10519000B9F08114A9F0B982DA820E94D1079C8308
:1051A0008B83F1E0FD8391E08C2D8A21811101C078
:1051B00090E09E8349815A816B817C818D8160DA88
:1051C000B394AA0C25E0B212E0CFF801C292D394B6
:1051D00038E0D312CECF0E94F60838C080918B02FF
:1051E000843021F110926D0228E130E060E40FB6C6
:1051F000F894A895209360000FBE6093600083B779
:10520000817F846083BF83B7816083BF78948895F2
:1052100083B78E7F83BF0FB6F894A8958091600006
:10522000886180936000109260000FBE0E94DC10C5
:10523000E1E8F2E08191811114C589E892E08E17CE
:105240009F07C1F774CF981391CF48DC8091A102DA
:10525000811509F465C0E0901004F0901104E11488
:10526000F10439F1C0901204D09013040E94D107C8
:105270008C010C191D09C7010E9436158017910772
:10528000C0F42091100430911104C9019927287F9E
:105290003327232B09F05BC144E0880F991F4A95FF
:1052A000E1F780579C4FDC0115962C9122FF0E945C
:1052B000B71080913D01811511F10091D00410913A
:1052C000D10401151105D9F00E94D107801B910B63
:1052D00020916304309164042817390780F4909179
:1052E000660480916504981709F434C11CD91092A2
:1052F0006404109263041092D1041092D00480913F
:105300008C03811569F00E94D10720918D033091A3
:105310008E03821B930B8F3F9F4710F40E949210C5
:1053200086E0ECE1F3E0DE01119601900D928A95A2
:10533000E1F7B0901D0310911E03D0901F03C090A1
:1053400020030091210310921E0310921F0310925C
:10535000200310922103812F8D29811509F441C06A
:10536000E0907A02F0907B020E94D1079C012E19F6
:105370003F0990911A03911509F46EC42531310546
:1053800080F19F3F19F09F5F90931A03111559F018
:105390000E94D30691E011160CF09FEF899F802D9B
:1053A000112480931E03D11459F00E94D30691E07A
:1053B0001D140CF09FEF899F802D112480931F03F3
:1053C00080911E03811569F0F0901F03F11449F0DC
:1053D0000E94C50680931E038F2D0E94C5068093F0
:1053E0001F038C2D802B811509F441C0E0907802B9
:1053F000F09079020E94D1079C012E193F099091EB
:105400001903911509F423C42135310580F19F3F1B
:1054100019F09F5F90931903C11459F00E94F3068D
:1054200091E01C140CF09FEF899F802D1124809334
:105430002003011559F00E94F30691E010160CF0BC
:105440009FEF899F802D1124809321038091200359
:10545000811569F0F0902103F11449F00E94C5060E
:10546000809320038F2D0E94C50680932103809195
:105470001D038B1119C080911E03811511F01813A3
:1054800013C020911F03211511F02D110DC0909113
:105490002103911511F0901307C0309120033111B1
:1054A00003C0822B892B81110E94060886E0FE0131
:1054B0003196ACE1B3E001900D928A95E1F70E943C
:1054C000430790917C02891721F080937C020E940F
:1054D000EA0880918B02843009F025CE83E0809326
:1054E000E9008091E80082FF1ECE8091E80090E004
:1054F00085FF0BC00E94980930E2E32EF12C8E014B
:105500000F5F1F4F8115C1F191E08091E8008B770B
:105510008093E800911509F406CE0091A90210913C
:10552000AA02E98101151105A9F1EE3F09F054C065
:105530008A81833020F08550833008F04DC0EA81A5
:10554000EE3008F049C0F0E0E753FD4C16C780E0AC
:1055500090E0A9CE0E944D221092D1041092D00466
:105560000E946106CCCE8091F100F80181938F01F9
:10557000F1E0EF1AF10841F28091E80085FDF3CFE8
:105580008091E8008B778093E8000E94980981154C
:1055900099F3BACFE43148F4E11549F0E150E33131
:1055A00030F4F0E0E952FD4CE8C6EE3F41F28FEFF7
:1055B000898312C01A8289E08B830EC08A8182306F
:1055C00081F08330B1F0813091F70E94EA08EBD688
:1055D0006B837C838D839E83CE0101960E94E809B4
:1055E000A2CD88E290E030D71B821C821D828E8380
:1055F000F3CF8091890290918A02892B69F388E028
:10560000E1E8F2E0DE01139601900D928A95E1F750
:10561000E3CF8A81823059F66B817C818D819E81B6
:10562000C2D688E290E02CD7D7CF4C816B818A819B
:105630000E940E139827892798279E838D83CCCFAD
:105640002D813E813227232732274C816B818A812D
:105650000E94700BC1CF0E941614BECF80E18A83D6
:10566000BBCF1A8287E8A8CF8C818D3108F0B4CFE8
:105670008A809B80982489249824A12CB12C9E0197
:105680002F5F3F4F79018901080F111DE016F106C8
:1056900009F4A2CF80E037E883169104A104B10495
:1056A00020F4C40187589C4FCFD6D70114968C9311
:1056B000BFEFEB1AFB0AEFEF8E1A9E0AAE0ABE0A84
:1056C000E5CF8091890290918A02892B09F484CFD9
:1056D0008C818D3108F080CF882E912CA12CB12C9B
:1056E000CA80DB80DC24CD24DC24E12CF12C8E016B
:1056F0000F5F1F4F412C512C3201481459046A048A
:105700007B0408F069CFF7E8CF16D104E104F10477
:1057100038F4D80114966C91C60187589C4FB0D6C6
:10572000BFEF4B1A5B0A6B0A7B0AEFEFCE1ADE0A59
:10573000EE0AFE0A0F5F1F4FE0CF21DB4DCF88E05E
:105740008ECF8C818D3108F047CF882E912CA12CE3
:10575000B12CCA80DB80DC24CD24DC24E12CF12CAC
:10576000412C512C32018E010B5F1F4F48145904FC
:105770006A047B0408F030CF80E0F0E8CF16F2E056
:10578000DF06E104F10418F4C60189965DD6D8015C
:105790008D938D01BFEF4B1A5B0A6B0A7B0AEFEF0B
:1057A000CE1ADE0AEE0AFE0AE1CF2C81022F10E0AB
:1057B0002D3108F011CF8A819B819827892798275E
:1057C0002C01612C712C8038F2E09F0708F004CF87
:1057D000822E912CA12CB12C40E852E060E070E0C8
:1057E0004419550966097709421751056105710584
:1057F00008F4F2CE2091890230918A02232B09F01D
:105800003EC01C0129E2220E311C80FBEE24FF2445
:10581000E0F880FF0BC0889617D69D8189279827CE
:10582000892781159C4711F48FEF8D83D501C40121
:10583000840D951DA61DB71D80FF19C0680161E08C
:10584000C61AD108CE0105968C0D9D1D9CA78BA76D
:10585000C101800F911FF8D5ABA5BCA59C91811506
:105860009C4721F48FEFEBA5FCA580838601FE0108
:105870003196EE0DFF1D2FEFE016F10638F08E0188
:105880000F5F1F4FC12CD12C760125C094818581DB
:1058900081159C4711F42483258362E0E60EF11CF8
:1058A0003296EACF70E8471672E057066104710439
:1058B00030F4D80114966C91C2018996E1D5BFEFFE
:1058C000CB1ADB0AEB0AFB0AEFEF4E1A5E0A6E0AEE
:1058D0007E0A0F5F1F4FC814D904EA04FB0410F3BB
:1058E0007BCE8091890290918A02892B09F474CE33
:1058F000CE0101960E94E809FFEF21EE34E0F1505D
:1059000020403040E1F700C00000F4CB88E0E2E541
:10591000F1E0DE01919601900D928A95E1F7FE018A
:1059200032968FE1DF011D928A95E9F786E089833F
:1059300088E07F96DE01159667CE84ED89831A8212
:105940001B821C8249CE8B819C81092E000CAA0BE4
:10595000BB0B25E0880F991FAA1FBB1F2A95D1F703
:10596000AC01BD01405E5F4F6F4F7F4F4817590735
:105970006A077B0708F430CE843D9105A105B10587
:1059800008F02ACE453D51056105710520F044ED32
:1059900050E060E070E0481B590BBC016E567B4F35
:1059A000CE0101961BD518CE4AE150E06FEF70E0B2
:1059B000CE01079632D58091890289830A831B82A2
:1059C0001C821D8281E013CE81E090E09093AA02B8
:1059D0008093A90282E390E09093800280937F02FB
:1059E0000E94D10790937E0280937D02F5CD011530
:1059F000110571F1D0908102E0907D02F0907E025D
:105A00000E94D1078E199F098536910540F1D1FE7C
:105A100026C0D0FE24C00E94D10790937E028093BE
:105A20007D0280917F029091800201979093800285
:105A300080937F02892B61F41092AA021092A9022E
:105A400081E090E090938A028093890200E010E068
:105A50008091890289830A8380917F02ADCD82E3A0
:105A600090E09093800280937F02F2CF10928A029E
:105A700010928902B1CD40E250E06FEF70E0CE01AC
:105A80000196CBD4A9CDEB81E93008F0A5CDF0E0AB
:105A9000E651FD4C72C4FE0133968DE1DF011D928B
:105AA0008A95E9F788E089838A838C8383E088A3D9
:105AB00093CD8C819AE0F92E8E010F5D1F4FF80176
:105AC000CF2C1192CA94E9F7B8010E94211589835D
:105AD000F801DE01129601900D92FA94E1F77CCD67
:105AE0001C818AE0FE013596DE01919601900D92AF
:105AF0008A95E1F789A19AA10E9401069AA389A338
:105B00008BA19CA10E9401069CA38BA38DA19EA1A9
:105B10000E9401069EA38DA38FA198A50E94010655
:105B200098A78FA38FEF183060F42AE0129FB0017E
:105B3000112467557D4F4AE050E0CE018196BED4D6
:105B400080E089830E940E0647CD2C816AE0CE0159
:105B50008196DC01E62F1D92EA95E9F7283080F462
:105B6000629FB001112467507D4F4AE050E05CD441
:105B700080E089838AE0FE01B196DE01129644CD71
:105B80008FEFF7CF1C818AE0FE013596DE019196FA
:105B900001900D928A95E1F789A59AA50E940106C8
:105BA0009AA789A78FEF183060F4FAE01F9FB00121
:105BB000112467507D4F4AE050E0CE0181967ED49B
:105BC00080E089830E949D1407CD2C8166E0CE0180
:105BD0008196DC01E62F1D92EA95E9F7283060F402
:105BE000629FB0011124675B7C4F46E050E01CD4FB
:105BF00080E0898386E0BFCF8FEFFBCF1C8186E0FA
:105C0000FE013596DE01919601900D928A95E1F79D
:105C100089A19AA10E9401069AA389A38BA19CA1A4
:105C20000E9401069CA38BA38FEF183060F4F6E06E
:105C30001F9FB0011124675B7C4F46E050E0CE010E
:105C400081963CD480E089830E94E114C5CC2B303E
:105C5000310508F0DECB0BCC2B30310508F093CBAF
:105C6000C0CB80916E02811509F461CA90E199BDA3
:105C7000A2E1A9BD09B400FEFDCF8091D8008F7DBF
:105C80008093D8008091E00082608093E000809152
:105C9000E00081FDFCCF0E94E40B49CA1F921FB6B1
:105CA0001F9211248F939F93AF93BF9380916D02A6
:105CB000811113C08091020290910302A09104020D
:105CC000B09105024196A11DB11D809302029093EF
:105CD0000302A0930402B0930502BF91AF919F917C
:105CE0008F911F901FBE1F90189578941F921FB61A
:105CF0001F9211248F939F93AF93BF9380910202C1
:105D000090910302A0910402B09105020196A11D99
:105D1000B11D8093020290930302A0930402B093FA
:105D20000502BF91AF919F918F911F901FBE1F9051
:105D300018951F920F920FB60F9211242F933F9335
:105D40004F935F936F937F938F939F93AF93BF9383
:105D5000EF93FF938091E10082FF09C08091E20000
:105D600082FF05C08091E1008B7F8093E1008091EC
:105D7000DA0080FF24C08091D80080FF20C080918D
:105D8000DA008E7F8093DA008091D90080FFA9C06D
:105D900080E189BD82E189BD09B400FEFDCF81E0CB
:105DA00080938B028091F101811109C00E94C90981
:105DB0000E943F0A8091E20084608093E20080911B
:105DC000E10080FF1AC08091E20080FF16C0809140
:105DD000E2008E7F8093E2008091E20080618093F8
:105DE000E2008091D80080628093D80019BC85E0E1
:105DF00080938B0283E0809303018091E10084FF14
:105E00002FC08091E20084FF2BC080E189BD82E138
:105E100089BD09B400FEFDCF8091D8008F7D8093AD
:105E2000D8008091E1008F7E8093E1008091E200B4
:105E30008F7E8093E2008091E20081608093E20097
:105E40008091F001811509F452C084E080938B02A7
:105E500080918B02843009F052C082E0809303016C
:105E60008091E10083FF2CC08091E20083FF28C075
:105E70008091E100877F8093E10082E080938B0234
:105E80001092F0018091E1008E7F8093E10080917B
:105E9000E2008E7F8093E2008091E2008061809337
:105EA000E20042E060E080E00E940F0A8091F00092
:105EB00088608093F00081E0809303018093020169
:105EC000FF91EF91BF91AF919F918F917F916F91D2
:105ED0005F914F913F912F910F900FBE0F901F90A8
:105EE000189519BC10928B021092F10168CF809125
:105EF000E30087FF02C083E0A9CF81E0A7CF81E064
:105F0000ADCF1F920F920FB60F921124EF92FF9216
:105F10000F931F932F933F934F935F936F937F93B1
:105F20008F939F93AF93BF93CF93EF93FF9309EE1C
:105F300010E0F8018081C091EC008F70C795CC27EC
:105F4000C795C82B108280EFE82EF12CF7018081D5
:105F5000877F808378940E941C0CF8011082F701DF
:105F6000808188608083CF70F801C083FF91EF91BA
:105F7000CF91BF91AF919F918F917F916F915F91E1
:105F80004F913F912F911F910F91FF90EF900F90A4
:105F90000FBE0F901F9018958EE1499B02C08A9505
:105FA000E1F7499BFECF0895599880E28A95F1F771
:105FB000599A0895FC013BE03A95F1F798E020E00A
:105FC00080E031E040E14A95F1F7880F499B02C03B
:105FD0008160232742E04A95F1F7000040E14A95AD
:105FE000F1F79A9579F790E19A95F1F799B132E046
:105FF0003A95F1F7000040E14A95F1F796959170D6
:1060000092272081920F90830895A1E0B0E0EAE00A
:10601000F0E375C119828C017C01E60EF11CBCDF36
:10602000CE010196C7DFF80181938F01EE15FF05C0
:10603000B1F781E09981911180E02196E6E07BC182
:10604000519A599A08955198599AE99AE9E6F0E0D7
:106050008081837F808308956150770B91E001C038
:10606000990F6A95EAF7692F90E021E0611108C065
:10607000911599F0599A80E28A95F1F75998089507
:10608000362F3823311539F0599A922730E23A9554
:10609000F1F76695EBCF5998F9CF5998ECCFFF926D
:1060A0000F931F93CF93DF93EC018C01060F111D0B
:1060B000F9907ADF68E08F2DCFDFC017D107C1F7E5
:1060C000CDB7DEB7E5E038C11F920F920FB60F9241
:1060D00011240F931F932F933F934F935F936F93CD
:1060E0007F938F939F93AF93BF93EF93FF93CF9340
:1060F000DF930F92CDB7DEB719824EDFCE01019646
:1061000059DF082F069506950695982F929595705C
:10611000202F2570920F292F237096959695920F18
:10612000982797708981892B811509F058C0043010
:1061300008F055C080E18A95F1F7599A519A82E0AA
:106140008A95F1F700C0599888E0089F80011124D2
:10615000D801AB5DBE4F1696ED91FC911797309725
:10616000A9F060916A0170916B0114962D913C9198
:106170001597260F371F11968D919C911297680FD6
:10618000791F13964C9113978C910995F801EB5D4B
:10619000FE4F6381611549F020916A0130916B01D6
:1061A00084819581820F931F7ADFFEDE80E18A95DC
:1061B000F1F759985198599A80E18A95F1F7F801C9
:1061C000EB5DFE4F6081611549F020916A013091CD
:1061D0006B0181819281820F931F17DFDDDE0F90AB
:1061E000DF91CF91FF91EF91BF91AF919F918F91EF
:1061F0007F916F915F914F913F912F911F910F91DF
:106200000F900FBE0F901F9018950F931F93CF9371
:10621000DF938C0104970CF05EC0F894519A599862
:1062200085E08A95F1F70000C02FC695C570802FD4
:106230008570C80F8C2F8370C695C69593E0000FAC
:10624000111F9A95E1F7C80FC8018C2BEC01ACDE49
:1062500000C068E08C2F00DF90E19A95F1F751982B
:10626000599A499B31C087E090E049992FC0F801C5
:10627000EB5DFE4F6381611559F020916A01309109
:106280006B0184819581820F931FBFDE811501F11F
:1062900083DE80E28A95F1F75998519A90E19A95B8
:1062A000F1F7F801EB5DFE4F6081611549F0209137
:1062B0006A0130916B0181819281820F931FEFDE21
:1062C00073DE789481E008C000C0CBCF019749F419
:1062D000519A599A789480E0DF91CF911F910F9154
:1062E000089500C0C2CF2F923F924F925F926F925B
:1062F0007F928F929F92AF92BF92CF92DF92EF9256
:10630000FF920F931F93CF93DF93CDB7DEB7CA1BD6
:10631000DB0B0FB6F894DEBF0FBECDBF09942A8801
:10632000398848885F846E847D848C849B84AA84A9
:10633000B984C884DF80EE80FD800C811B81AA8136
:10634000B981CE0FD11D0FB6F894DEBF0FBECDBF01
:10635000ED01089597FB072E16F4009406D077FD03
:1063600008D028D007FC05D03EF4909581959F4F2A
:106370000895709561957F4F0895EE0FFF1F05906A
:10638000F491E02D0994082E817006940694811DE5
:106390000694811D0694811D0694811D0694811D1D
:1063A0000694801D089569279627692778278727EF
:1063B00078270895AA1BBB1B51E107C0AA1FBB1F6A
:1063C000A617B70710F0A61BB70B881F991F5A9581
:1063D000A9F780959095BC01CD010895FB01DC01E2
:1063E00002C005900D9241505040D8F70895FB012E
:1063F000DC0104C08D910190801921F4415050407E
:10640000C8F7881B990B0895FB01DC0102C00190BD
:106410000D9241505040D8F70895DC0101C06D93B2
:1064200041505040E0F70895DC01CB01FC01F9999F
:10643000FECF06C0F2BDE1BDF89A319600B40D92D0
:1064400041505040B8F70895F999FECF92BD81BDF3
:10645000F89A992780B50895A8E1B0E042E050E0AD
:10646000E5CFDC01A40FB51F4150504040F0CB01F7
:10647000840F951F2E9105D041505040D8F70895B4
:10648000262FF999FECF92BD81BDF89A019700B4ED
:10649000021639F01FBA20BD0FB6F894FA9AF99A8D
:1064A0000FBE08950396272FECDFEADF252FE9DFE3
:1064B000242FE7CF0196272FE4DFE2CFDC01CB01C9
:1064C00002C02D9105D041505040D8F70895262F95
:1064D000F999FECF1FBA92BD81BD20BD0FB6F894C9
:1064E000FA9AF99A0FBE01960895F894FFCF3B08E7
:1064F00040084208470857085708570857085708E0
:1065000057085708570849084D08500855086508A6
:106510006B086F08F90C1F0D250D1F0D250D770D4C
:10652000980D250D9E0EAB0EC61B2E1CCE1B981B68
:106530009C1BD21BA01BD61BE21BAC1B271CB01B39
:10654000E61BB41BEA1B0F1CB81BEE1B161CBE1B64
:10655000F41BFC1BA41BDA1BA81BDE1BC21BF81BB5
:10656000061C1F1C251C921BCA1B351C641B6A1BA6
:10657000561B5E1B701B761B7C1B8E1D8E1DC51D46
:10658000C51D761E911EE91DE91D961E091F1A1FC5
:106590001A1F862C9D2CA32CEC2AEC2AD42CE42C3C
:1065A000F72C362D3B2DEC2AEC2AEC2A432DDA2A47
:1065B000DE2A092B152B202B2B2BD72AD72AD72ABB
:1065C000D72A712C2E2B312B342B612B9D2B9F2BFB
:1065D000A12BD52B4B2D592D702DA52DC22DEC2A7D
:0665E000EC2AE52DFE2D62
:1065E600000001006692F732F49790F633F5C694F0
:1065F6009331363435FFFFFF01CE07FA0A1F091023
:106606000B150BF10A00000001000000000000005D
:106616000401000000040500000000000001F4323F
:10662600F79266F533F6909736319394C63534FF74
:10663600FFFF76319764334BC0A60044227B4901A5
:106646002701AC004F02680288029002E200E900CE
:10665600EA00B500B600B700CD008301CC008A0180
:106666009201940121022302240225022602270216
:106676002A02B300B4006F0070009F01CB019F0295
:10668600A002E200E900EA00B500B600B700CD00BE
:106696008301CC008A019201940121022302240283
:1066A6002502260227022A02B300B4006F007000FA
:0866B6009F01CB019F02A0022D
:00000001FF
